:100000000C94340018950000189500001895000015
:10001000189500001895000018950000189500002C
:10002000189500001895000018950000189500001C
:10003000189500001895000018950000189500000C
:1000400018950000189500001895000018950000FC
:1000500018950000189500001895000018950000EC
:1000600018950000189500008FEF8DBFC0ECE8E5F3
:100070004E2E84E08EBFD4E0F4E05F2EEEEFF3E08E
:10008000A0E0B1E088278D933197E9F7662488EEE8
:1000900093E00E94B30C87E48093000184E780938F
:1000A000010180E78093020181EC85B98EE384B978
:1000B00080EF88B98CE087B987E98BB988E68AB97F
:1000C0000E94C20C80E08093B90080E28093B80067
:1000D00086E080937A0083E080937E000027A9E287
:1000E000B0E08C9180FB0EF401E041E0041711F0C8
:1000F0000C947F0081EA80931A010C94820081EFB6
:1001000080931A01AAE1B1E08C9184BD83E085BDA2
:1001100080E086BD80E087BD80E088BDAAE1B1E0D7
:100120008C918093800083E08093810080E08093B5
:10013000850080E08093840080E08093870080E0E9
:100140008093860080E08093890080E0809388001F
:1001500080E080938B0080E080938A0080E0809331
:10016000B600AAE1B1E08C918093B00084E0809366
:10017000B10080E08093B20080E08093B30080E023
:100180008093B40082E390E00E94B30C83E08A93F2
:1001900012E4A0E0B1E00E94120D84E690E00E941B
:1001A000B30CE7E0F0E0ACE2B1E00E948C0DE9E0D6
:1001B000F0E0AEE2B1E00E948C0DEBE0F0E0A0E3F5
:1001C000B1E00E948C0DEDE0F0E0A4E3B1E00E940C
:1001D0008C0DEFE0F0E0A6E3B1E00E948C0DE1E1D0
:1001E000F0E0A8E3B1E00E948C0DAEE2B1E00D9129
:1001F0001C91A0E3B1E04D915C91041B150BA2E3AF
:10020000B1E00D931C93A6E3B1E00D911C91A8E31E
:10021000B1E04D915C91041B150BAAE3B1E00D9385
:100220001C9300E918E527E130E0A2E3B1E04D912D
:100230005C91662777270E94560CA0E2B1E04D93AF
:100240005D936D937D93A0E2B1E08D919C91ACE3C1
:10025000B1E08D939C9300E918E527E130E0AAE333
:10026000B1E04D915C91662777270E94560CA0E281
:10027000B1E04D935D936D937D93A0E2B1E08D91DC
:100280009C91AEE3B1E08D939C9308E114EE23E0E2
:1002900030E0A2E3B1E04D915C91662777270E94A0
:1002A000560CA0E2B1E04D935D936D937D93A0E277
:1002B000B1E08D919C91A0E4B1E08D939C930E945C
:1002C000A90986B5A4E2B1E08D9388278C930E949A
:1002D000850A00910301003011F00C9473010E9413
:1002E000D0010C94850100910301013011F00C94B0
:1002F0007D010E94E7020C94850100910301023008
:1003000011F00C9485010E94D6032698A0E1B1E07B
:100310009C9195FF04C01E9B10C09F7D9C931E99CD
:100320000CC08EE19F9399270E94B30C9F911E9958
:1003300004C090629C930E9499052798A0E1B1E0C7
:100340009C9194FF04C01F9B10C09F7E9C931F999B
:100350000CC08EE19F9399270E94B30C9F911F9927
:1003600004C090619C930E94AB050027A6E2B0E018
:100370008C9186FB0EF401E040E0041711F00C9420
:10038000C3010C94C5010C94690184E690E00E94BD
:10039000B30CA6E2B0E08C9186FBDEF70C94EA0A7F
:1003A0000E94530A0E94660A81E090E00E94B30C0A
:1003B000ACE2B1E00D911C914FE050E0040F151F2D
:1003C000ABE1B1E00D931C93ABE1B1E04D915C91D9
:1003D000A8E2B1E00D911C910417150718F011F077
:1003E0000C94F4010C94F701429A0C94F801429891
:1003F000ACE2B1E00D911C914FE050E0041B150BF5
:10040000ABE1B1E00D931C93ABE1B1E04D915C9198
:10041000A8E2B1E00D911C910417150710F00C949F
:1004200014022D9A0C9415022D98A4E3B1E00D91BD
:100430001C914FE050E0040F151FABE1B1E00D93AC
:100440001C93ABE1B1E04D915C91AAE2B1E00D915A
:100450001C910417150718F011F00C9431020C943C
:1004600034022C9A0C9435022C98A4E3B1E00D913F
:100470001C914FE050E0041B150BABE1B1E00D9374
:100480001C93ABE1B1E04D915C91AAE2B1E00D911A
:100490001C910417150710F00C945102439A0C9408
:1004A00052024398A6E2B1E00D911C914CED55E04B
:1004B000040F151FABE1B1E00D931C93ABE1B1E06C
:1004C0000D911C910F305EE0150718F011F00C949F
:1004D0006B020C947702ABE1B1E00D911C9140E10D
:1004E0005EE0041B150BABE1B1E00D931C9309EA30
:1004F00011E020E030E0ABE1B1E04D915C91662786
:1005000077270E94420DA0E2B1E00D931D932D9339
:100510003D93A0E2B1E00D911D912D913C9148EEEB
:1005200053E060E070E00E94560CA0E2B1E04D9311
:100530005D936D937D93A0E2B1E08D919C91A3E1D9
:10054000B1E08D939C93A3E1B1E00D911C914DEF2F
:1005500052E0040F151FA1E1B1E00D931C93A1E13E
:10056000B1E00D911C91093F55E0150718F011F00D
:100570000C94BC020C94C802A1E1B1E00D911C9155
:100580004AEF55E0041B150BA1E1B1E00D931C935C
:100590005A924A9281E0A42DB52D8C9381E00E945D
:1005A000F40B0E94E508229681E00E94F00B5A921B
:1005B0004A9282E0A42DB52D8C9381E00E94F40B29
:1005C0000E94E508229681E00E94F00B08950E94A7
:1005D000530A81E090E00E94B30CA0E3B1E04D919A
:1005E0005C91A8E2B1E00D911C910417150718F079
:1005F00011F00C94030380E090E0ABE1B1E08D9347
:100600009C930C941103A8E2B1E00D911C91A0E31E
:10061000B1E04D915C91041B150BABE1B1E00D9382
:100620001C93ACE3B1E00D911C9122273327ABE181
:10063000B1E04D915C91662777270E94420DA0E2C0
:10064000B1E00D931D932D933D93A0E2B1E00D9188
:100650001D912D913C9148EE53E060E070E00E94C6
:10066000560CA0E2B1E04D935D936D937D93A0E2B3
:10067000B1E08D919C91A3E1B1E08D939C93A3E1B6
:10068000B1E00D911C910A3F55E0150718F011F0EB
:100690000C944C030C9452038AEF95E0A3E1B1E073
:1006A0008D939C93A8E3B1E04D915C91AAE2B1E0F7
:1006B0000D911C910417150718F011F00C946803A4
:1006C00080E090E0ABE1B1E08D939C930C947603D5
:1006D000AAE2B1E00D911C91A8E3B1E04D915C91CB
:1006E000041B150BABE1B1E00D931C93AEE3B1E03D
:1006F0000D911C9122273327ABE1B1E04D915C9124
:10070000662777270E94420DA0E2B1E00D931D936A
:100710002D933D93A0E2B1E00D911D912D913C915F
:1007200048EE53E060E070E00E94560CA0E2B1E0B9
:100730004D935D936D937D93A0E2B1E08D919C917B
:10074000A1E1B1E08D939C93A1E1B1E00D911C91E9
:100750000A3F55E0150718F011F00C94B1030C9402
:10076000B7038AEF95E0A1E1B1E08D939C935A9293
:100770004A9281E0A42DB52D8C9381E00E94F40B68
:100780000E94E508229681E00E94F00B5A924A925C
:1007900082E0A42DB52D8C9381E00E94F40B0E9481
:1007A000E508229681E00E94F00B08950027A0E161
:1007B000B1E08C9187FB0EF401E040E0041781E08A
:1007C00009F080E08F934091080100910A0104171D
:1007D00081E008F480E09F918923882311F40C9430
:1007E0002E04EEE0F1E0FA93EA935A924A92A4E0E2
:1007F000B1E08D919C91A42DB52D8D939C9382E0B9
:100800000E94F40B5A924A9280910C01A42DB52DAE
:100810008C9381E00E94F40B5A924A9281E0A42DBD
:10082000B52D8C9381E00E94F40B0E94B9062896A6
:1008300084E00E94F00BA4E0B1E00E94F80B00916C
:100840000E01013011F00C942B0480E090E0A4E044
:10085000B1E08D939C9381E080930A010027A0E191
:10086000B1E08C9186FB0EF401E040E0041781E0DA
:1008700009F080E08F934091090100910B0104176A
:1008800081E008F480E09F918923882311F40C947F
:100890008604EFE0F1E0FA93EA935A924A92A6E0D6
:1008A000B1E08D919C91A42DB52D8D939C9382E008
:1008B0000E94F40B5A924A9280910D01A42DB52DFD
:1008C0008C9381E00E94F40B5A924A9282E0A42D0C
:1008D000B52D8C9381E00E94F40B0E94B9062896F6
:1008E00084E00E94F00BA6E0B1E00E94F80B0091BA
:1008F0000F01013011F00C94830480E090E0A6E039
:10090000B1E08D939C9381E080930B010027A0E1DF
:10091000B1E08C9187FB0EF401E040E0041711F088
:100920000C949704AAE0B1E08C918F5F8C930091B6
:100930000A01003011F00C94A00481E080930A01B8
:100940000027A0E1B1E08C9186FB0EF401E040E0CD
:10095000041711F00C94B104ABE0B1E08C918F5FFF
:100960008C9300910B01003011F00C94BA0481E0DB
:1009700080930B010E94530A00911501003011F081
:100980000C94E004A6E3B1E00D911C9144E650E024
:10099000041B150BABE1B1E00D931C93ABE1B1E08F
:1009A0004D915C91AAE2B1E00D911C9104171507DD
:1009B00010F00C94DE0481E0809315010C94FE0489
:1009C000A6E3B1E00D911C9148E250E0041B150B29
:1009D000ABE1B1E00D931C93ABE1B1E04D915C91C3
:1009E000AAE2B1E00D911C910417150718F011F05F
:1009F0000C94FC040C94FE040E948B0600911601DA
:100A0000003011F00C942505A8E3B1E00D911C9184
:100A100044E650E0040F151FABE1B1E00D931C93C9
:100A2000ABE1B1E04D915C91AAE2B1E00D911C9176
:100A30000417150718F011F00C9420050C942305E9
:100A400081E0809316010C944005A8E3B1E00D917C
:100A50001C9148E250E0040F151FABE1B1E00D938B
:100A60001C93ABE1B1E04D915C91AAE2B1E00D9134
:100A70001C910417150710F00C9440050E94A20663
:100A80000027A0E1B1E08C9187FB0EF401E041E08A
:100A9000041711F00C944F052C9A0C9450052C98C7
:100AA0000027A0E1B1E08C9186FB0EF401E041E06B
:100AB000041711F00C945F05439A0C946005439859
:100AC0005798A0E1B1E09C9193FF04C04F9B10C0E8
:100AD000977F9C934F990CC08EE19F9399270E941A
:100AE000B30C9F914F9904C098609C930E94B405E9
:100AF0002098A0E1B1E09C9192FF04C0189B10C027
:100B00009B7F9C9318990CC08EE19F9399270E941C
:100B1000B30C9F91189904C094609C930E9407069F
:100B2000EF93FF93ECECF7E00E94AA0CFF91EF919A
:100B3000089586B5A4E2B1E08D9388278C93A3E055
:100B4000B1E08C918F5F8C932D98429843982C98AC
:100B50000E94850A089586B5A4E2B1E08D938827A6
:100B60008C930E941C0A089586B5A4E2B1E08D938F
:100B700088278C930027A0E1B1E08C9187FB0EF4CD
:100B800001E040E0041711F00C94E00580E090E0F3
:100B9000A4E0B1E08D939C9381E080930A01ACE0E6
:100BA000B1E08C918F5F8C9300910C01073018F0AD
:100BB00011F00C94DD050C94E00580E080930C01AD
:100BC0000027A0E1B1E08C9186FB0EF401E040E04B
:100BD000041711F00C94060680E090E0A6E0B1E066
:100BE0008D939C9381E080930B01ADE0B1E08C91FB
:100BF0008F5F8C9300910D01073018F011F00C9469
:100C000003060C94060680E080930D01089586B5D6
:100C1000A4E2B1E08D9388278C93A0E3B1E04D91DD
:100C20005C91A8E2B1E00D911C910417150718F032
:100C300011F00C94230680E090E0ABE1B1E08D93DD
:100C40009C930C943106A8E2B1E00D911C91A0E3B5
:100C5000B1E04D915C91041B150BABE1B1E00D933C
:100C60001C93A0E4B1E00D911C9122273327ABE146
:100C7000B1E04D915C91662777270E94420DA0E27A
:100C8000B1E00D931D932D933D93A0E2B1E00D9142
:100C90001D912D913C9148EE53E060E070E00E9480
:100CA000560CA0E2B1E04D935D936D937D938091DE
:100CB000200180931A0100911A01003011F00C9468
:100CC000640681E080931A010027A0E1B1E08C91D5
:100CD00087FB0EF401E040E0041711F00C94770656
:100CE00081E080930A0180911A0180930801002716
:100CF000A0E1B1E08C9186FB0EF401E040E0041726
:100D000011F00C948A0681E080930B0180911A0106
:100D100080930901089586B5A4E2B1E08D938827F8
:100D20008C93A0E1B1E08C9187FB882780F98095B6
:100D300080FBA0E1B1E08C9187F98C9380E08093F7
:100D40001501089586B5A4E2B1E08D9388278C93B0
:100D5000A0E1B1E08C9186FB882780F9809580FB2B
:100D6000A0E1B1E08C9186F98C9380E0809316012C
:100D70000895A881B981AD90BB24AFE0B1E0AA0C81
:100D8000BB1CAA0DBB1D8D919C91A8E1B1E08D9378
:100D90009C93AA81BB810C91003011F00C94EE065B
:100DA000AC81BD818D919C91A8E1B1E08D939C9324
:100DB000AC81BD810D911C91093F55E0150710F4E0
:100DC0000C94E80681E0AE81BF818C930C94EC0614
:100DD00080E0AE81BF818C930C94C308AA81BB8153
:100DE0000C91013011F00C94170709EF15E0AC815C
:100DF000BD814D915C91041B150BA8E1B1E00D93F1
:100E00001C93AC81BD810D911C91093F55E01507E4
:100E100010F40C94110781E0AE81BF818C930C9487
:100E2000150780E0AE81BF818C930C94C308AA8122
:100E3000BB810C91023011F00C945407AC81BD8140
:100E40000D911C910A3F55E0150710F00C943207E4
:100E5000AC81BD818D919C91A8E1B1E08D939C9373
:100E60000C943E0704EF1BE0AC81BD814D915C9179
:100E7000041B150BA8E1B1E00D931C93AC81BD815F
:100E80000D911C91033F5BE0150710F40C944E0785
:100E900081E0AE81BF818C930C94520780E0AE81DB
:100EA000BF818C930C94C308AA81BB810C91033041
:100EB00011F00C94D107AC81BD810D911C91083CBF
:100EC00050E0150710F00C946D0780E090E0A8E169
:100ED000B1E08D939C930C94BB07AC81BD810D91C7
:100EE0001C91003951E0150710F00C947F078FEF2B
:100EF00090E0A8E1B1E08D939C930C94BB07AC818A
:100F0000BD810D911C91083552E0150710F00C942D
:100F100091078EEF91E0A8E1B1E08D939C930C9442
:100F2000BB07AC81BD810D911C91003253E01507C8
:100F300010F00C94A3078DEF92E0A8E1B1E08D933F
:100F40009C930C94BB07AC81BD810D911C91083E14
:100F500053E0150710F00C94B5078CEF93E0A8E16F
:100F6000B1E08D939C930C94BB078BEF94E0A8E1C8
:100F7000B1E08D939C93AC81BD810D911C910F3A92
:100F800054E0150710F40C94CB0781E0AE81BF81CB
:100F90008C930C94CF0780E0AE81BF818C930C942E
:100FA000C308AA81BB810C91043011F00C940F0886
:100FB000AC81BD818D919C91A8E1B1E08D939C9312
:100FC000A8E1B1E00D911C910E3F51E0150718F01A
:100FD00011F00C94ED070C94F9070CEF13E0A8E165
:100FE000B1E04D915C91041B150BA8E1B1E00D93AC
:100FF0001C93AC81BD810D911C910B3F53E01507F3
:1010000010F40C94090881E0AE81BF818C930C949C
:101010000D0880E0AE81BF818C930C94C308AA8137
:10102000BB810C91053011F00C945108AC81BD814D
:101030000D911C914EEF51E0040F151FA8E1B1E096
:101040000D931C93A8E1B1E00D911C910C3F53E06E
:10105000150718F011F00C942F080C943B0808EFBA
:1010600017E0A8E1B1E04D915C91041B150BA8E1DC
:10107000B1E00D931C93AC81BD810D911C910B3F90
:1010800053E0150710F40C944B0881E0AE81BF814A
:101090008C930C944F0880E0AE81BF818C930C94AC
:1010A000C308AA81BB810C91063011F00C949308FF
:1010B000AC81BD810D911C914CEF53E0040F151FC5
:1010C000A8E1B1E00D931C93A8E1B1E00D911C9152
:1010D0000A3F55E0150718F011F00C9471080C94B4
:1010E0007D0804EF1BE0A8E1B1E04D915C91041B89
:1010F000150BA8E1B1E00D931C93AC81BD810D915E
:101100001C910B3F53E0150710F40C948D0881E0FF
:10111000AE81BF818C930C94910880E0AE81BF8139
:101120008C930C94C308AA81BB810C91073011F0F9
:101130000C94C308AC81BD810D911C91003050E02E
:10114000150711F00C94AF088AEF95E08A939A93F3
:101150000E94FF0B2296A8E1B1E00D931C93AC8195
:10116000BD810D911C91073C50E0150710F40C94C3
:10117000BF0881E0AE81BF818C930C94C30880E0EE
:10118000AE81BF818C93A8E1B1E08D919C91A88143
:10119000B981AD90BB24AFE0B1E0AA0CBB1CAA0D95
:1011A000BB1D8D939C935A924A92AA81BB818C91CC
:1011B000A42DB52D8C9381E00E94F40B0E94E508CC
:1011C000229681E00E94F00B0895A881B981AD902C
:1011D000BB24AFE0B1E0AA0CBB1CAA0DBB1D8D91D6
:1011E0009C91A8E1B1E08D939C93A8E1B1E00D91B1
:1011F0001C910F3F50E0150710F00C940B098FEF76
:1012000080931D018091180180931E0180E08093DE
:101210001F010C947C09A8E1B1E00D911C910E3FD7
:1012200051E0150710F00C9424090EEF40911801BD
:10123000041BADE1B1E00C938FEF80931E0180E0C1
:1012400080931F010C947C09A8E1B1E00D911C91E1
:101250000D3F52E0150710F00C943D0980E080939B
:101260001D018FEF80931E01009118014EEF041BAA
:10127000AFE1B1E00C930C947C09A8E1B1E00D91D1
:101280001C910C3F53E0150710F00C94560980E0B8
:1012900080931D010CEF40911801041BAEE1B1E0F9
:1012A0000C938FEF80931F010C947C09A8E1B1E0AF
:1012B0000D911C910B3F54E0150710F00C946F0931
:1012C000009118014CEF041BADE1B1E00C9380E0FC
:1012D00080931E018FEF80931F010C947C098FEF88
:1012E00080931D0180E080931E010AEF4091180158
:1012F000041BAFE1B1E00C93A881B9810C910130DE
:1013000011F00C949309ADE1B1E08C9187BDAEE191
:10131000B1E08C9180938800AFE1B1E08C91809333
:10132000B3000C94A809A881B9810C91023011F086
:101330000C94A809ADE1B1E08C9188BDAEE1B1E0BB
:101340008C9180938A00AFE1B1E08C918093B400DE
:101350000895E1E0F0E0A3E0B1E00E948A0DE2E050
:10136000F0E0ACE0B1E00E948A0DE3E0F0E0ADE037
:10137000B1E00E948A0DE4E0F0E0A8E0B1E00E9454
:101380008A0DE5E0F0E0A9E0B1E00E948A0DE6E018
:10139000F0E0A0E1B1E00E948A0D0091030102306B
:1013A00018F011F00C94D6090C94D90980E08093C0
:1013B000030100910C01073018F011F00C94E209C0
:1013C0000C94E50980E080930C0100910D01073039
:1013D00018F011F00C94EE090C94F10980E0809360
:1013E0000D0100910801003011F00C94FA0981E020
:1013F0008093080100910901003011F00C94030A58
:1014000081E08093090180E090E0A4E0B1E08D9359
:101410009C9380E090E0A6E0B1E08D939C9381E006
:1014200080930A0181E080930B0180E08093150195
:1014300080E0809316010895E1E0F0E0A3E0B1E0E0
:101440007BE70E94790DE2E0F0E0ACE0B1E07BE701
:101450000E94790DE3E0F0E0ADE0B1E07BE70E94AF
:10146000790DE4E0F0E0A8E0B1E07BE70E94790DBF
:10147000E5E0F0E0A9E0B1E07BE70E94790DE6E06D
:10148000F0E0A0E1B1E07BE70E94790D2D9A429A4D
:10149000439A2C9A88EE93E00E94B30C2D984298C0
:1014A00043982C98089580E080937C000E94650DFD
:1014B000A8E2B1E08D939C9381E080937C000E9430
:1014C000650DAAE2B1E08D939C93089581E4809329
:1014D000000181E08A9312E4A0E0B1E00E94120DC5
:1014E0008AE090E00E94B30C22E480E092E0A6E261
:1014F000B1E00E941B0D009126018091270180938D
:101500002601A7E2B1E00C93089500910301023097
:1015100018F011F00C948E0A0C94910A80E08093DC
:10152000030100910301003011F00C94B30A2D9ACD
:10153000429A439A2C9A84EF91E00E94B30C2D9822
:10154000429843982C988FE48093000181E08A931D
:1015500012E4A0E0B1E00E94120D8AE090E00E9447
:10156000B30C0C94E90A00910301013011F00C94C2
:10157000C30A2D9A429A84EF91E00E94B30C2D98F1
:1015800042980C94E90A00910301023011F00C9486
:10159000E90A439A2C9A84EF91E00E94B30C439895
:1015A0002C9880E090E0A4E0B1E08D939C9380E0E3
:1015B00090E0A6E0B1E08D939C9381E080930A01D6
:1015C00081E080930B0180E08093150180E080939F
:1015D0001601089584E690E00E94B30C80E08093A9
:1015E0001A01439A2C982D98429880E08093170115
:1015F0000E94530A8AE090E00E94B30C3E98A0E15A
:10160000B1E09C9191FF04C0369B10C09D7F9C93DC
:1016100036990CC08EE19F9399270E94B30C9F913D
:10162000369904C092609C930E94730B009117013D
:10163000013011F00C941E0B0C94200B0C94F80A42
:1016400084E690E00E94B30C83E48093000181E083
:101650008A9312E4A0E0B1E00E94120D82E390E0D0
:101660000E94B30C81E080931A0100911A010630A8
:1016700018F011F00C945E0B439A2C982D98429818
:1016800084EC99E00E94B30C4398429A84EC99E070
:101690000E94B30C42982C9A84EC99E00E94B30CFF
:1016A0002C982D9A84EC99E00E94B30CAAE1B1E049
:1016B0008C918F5F8C9310F40C94350B85E48093A0
:1016C000000181E08A9312E4A0E0B1E00E94120DD3
:1016D00082E390E00E94B30C439A2C9A2D9A429A8E
:1016E00000000C94700B88EE93E00E94B30C00276E
:1016F000A6E2B0E08C9186FB0EF401E040E0041716
:1017000011F00C94880B81E0809317010C94DE0B90
:1017100000911A01003011F00C94990BE1E1F0E016
:10172000AAE2B1E07BE70E947B0D43982C9A0C94CF
:10173000DE0B00911A01013011F00C94AA0BEFE0BE
:10174000F0E0AAE2B1E07BE70E947B0D2C982D9A95
:101750000C94DE0B00911A01023011F00C94BB0BBB
:10176000EBE0F0E0A8E2B1E07BE70E947B0D2D9872
:10177000429A0C94DE0B00911A01033011F00C9484
:10178000CD0BE9E0F0E0A8E2B1E07BE70E947B0D41
:10179000439A2C9A2D9A0C94DE0BEDE0F0E0AAE22D
:1017A000B1E07BE70E947B0DE7E0F0E0A8E2B1E06A
:1017B0007BE70E947B0D2C982D984298AAE1B1E01E
:1017C0008C918F5F8C9300911A01043018F011F006
:1017D0000C94EC0B0C94EF0B80E080931A010895AD
:1017E000481A8827580A0895480E8827581E0895D1
:1017F000ED91FC91EF5FFF4FFC93EE9308954091C4
:101800004201509143010DE815E30E94130C49E198
:1018100056E3040F151F00934201109343014981C1
:1018200058810C94390C09D00E94380D00FC10D05E
:10183000089503D01ED001F8F9CF0024E89457FF93
:1018400002C009D0689400F80BD010F80124089564
:1018500002D009D00895509540954F5F5F4F08958D
:10186000E89417FF0895009510950F5F1F4F689437
:101870000895352F242FE894452B11F4689408958A
:10188000512F402F0027112780E1440F551F001FC3
:10189000111F021B130B416018F4020F131F4E7F20
:1018A0008A9599F7089500FC05D0089530D005D0A9
:1018B00001F8F9CF37D03FD00895842F952FA62F68
:1018C000B72FE894452B462B472B11F468940895C5
:1018D000402F512F622F732F0027112722273327E4
:1018E000F0E2440F551F661F771F001F111F221FB4
:1018F000331F081B190B2A0B3B0B416028F4080F00
:10190000191F2A1F3B1F4E7FFA9559F7089500248F
:10191000E89477FF02C006D0689400F809D010F868
:101920000124089512D04F5F5F4F6F4F7F4F08958E
:10193000E89437FF089500951095209530950F5F36
:101940001F4F2F4F3F4F68940895409550956095D5
:10195000709508953197F1F70895689462F80895A5
:10196000E89462F80895EF93FF93EE27E82BE92BB4
:1019700031F0E0EDF7E03197F1F70197D1F7FF9102
:10198000EF910895449A459A3C983D98089568943B
:101990004093BC008F939F9388279927019629F045
:1019A0004091BC0047FFFACFE8949F918F9162F875
:1019B000089544EAECCF44E94093BC004091BC0058
:1019C00047FDFCCF08951093BB0044E8E0DF8F9300
:1019D0009F9388279927019671F04091B900487F1D
:1019E000483FC9F3E894483139F0483229F040348F
:1019F00019F0403509F068949F918F9162F808952D
:101A000044E801C044ECC3DF1091BB004091B90031
:101A1000487F483FD9F326F06894487009F0E8946D
:101A200062F80895C6DF1E7FCEDF89911D91CBDF5E
:101A30008A95E1F7C0CF122F803059F0BADF1E7FB0
:101A4000C2DFAF93BF931D91BEDF8A95E1F7BF91CF
:101A5000AF91AFDF903059F0122F1160B4DF9130A9
:101A600011F4CEDF01C0CEDF1D939A95C1F7A3CF4D
:101A70000F92B801469F8001479F100D569F100D91
:101A80000F9008950F921F922F92C801D901489F7D
:101A900080014A9F90014B9F202C499F100D211DD2
:101AA000321D5A9F202C589F100D211D321D599F09
:101AB000200D311D689F200D311D699F300D789FCD
:101AC000300D2F901F900F90089580917A00806CB8
:101AD00080937A0080917A0086FDFCCF8091780017
:101AE000909179000895F999FECFE1BDF2BD31964C
:101AF000089591E001C092E07B3751F47FB7F894EC
:101B0000F2DF8D9180BDFA9AF99A9A95C9F77FBF55
:101B10007727089591E001C092E0E5DFF89A80B55B
:081B20008D939A95D1F7089509
:00000001FF
